:1000000013C0189518951895189518951895189562
:100010001895189518951895189518951895189578
:1000200018951895189518958FE181BD87E181BDC8
:100030008FE58DBFC6E5EAE44E2E84E08EBFD4E0A6
:10004000F4E05F2EEEEFF3E0A0E6B0E088278D93BA
:100050003197E9F766248FEF84BBA89A80E991E095
:1000600010D0A89888EC90E00CD0F7CFF894FFCF90
:100070003197F1F70895689462F80895E89462F86A
:100080000895EF93FF93EE27E82BE92B31F0EAEF89
:10009000F0E03197F1F70197D1F7FF91EF910895D3
:00000001FF
